:105C0000AA550013FFFFFFFFFFFFFFFFFFFFFFFF8E
:105C1000B0126C74B090E1071EC5022C22C3304153
:105C2000B240805A5C01804328C7C043E6C3F040BD
:105C30000700E1C3C043DEC3F0405E00D9C3B01229
:105C4000188380439CC4804390C4F2D08000020239
:105C5000B04020009CC4B0C000087EC4B0B00008B2
:105C600078C4FC27804376C4B0C080016CC4B0D037
:105C7000800066C41F408EBB3FF07F00B01260669C
:105C8000B0121A66B040409C62C4B0C000044AC45E
:105C900005430443C04376C3F04398C38043C2C660
:105CA0008043C0C6A0B332C4FD27A0C32CC4B01229
:105CB000F65FB0B00F0026C4052434905E01022CBC
:105CC00034405E01B0127264B0B000040CC4092408
:105CD000B0C0802104C4B0D00040FEC3804382C65F
:105CE0001B3CC0934EC303241553C04346C31453F7
:105CF0003490FA00032C8043F4C3D43F3490F40171
:105D0000D12BB0C08021D2C3B0D00040CCC38043DF
:105D100050C635900A00002CB012E064B0B00040CC
:105D2000B8C3F723B0C08001B0C3B0D00001AAC38C
:105D3000C04320C6B090AC0DB4C3022CF04314C6CF
:105D40001F40C2BA3FF07F00B0126066B0121A6600
:105D50008043AEC3B0403200ACC305430443C043EC
:105D6000ACC28043FCC58043FAC5B0C00F006EC30F
:105D7000B040409C76C3B0C000045EC3B0B0030026
:105D80005CC32520B0127264B0B000044CC3E020A4
:105D9000A0B346C3F327A0C340C3B012F65FC093BD
:105DA0006CC2092014533490F401E82B90D33AC309
:105DB000B012D25ECD3CC04354C2C09376C2DE273F
:105DC00015533590C800DA2BA0D31EC3CD3CB0C00C
:105DD000802106C3B0D0004000C3804384C5B01208
:105DE000E064B0B00040F2C2FA23B0C00C00EEC2D2
:105DF000B0C08001E4C2B0D08000DEC21F4006BA4D
:105E00003FF07F00B0126066B0121A66B040409C4E
:105E1000DAC2B0C00004C2C205430443C043EEC1AD
:105E2000F04310C2B0B00C00B4C22520B0127264AE
:105E3000B0B00004A4C28C20A0B39EC2F327A0C3BC
:105E400098C2B012F65FC093C4C1092014533490B5
:105E5000F401E82B90D392C2B012D25E793CC043D9
:105E6000ACC1C093CEC1DE2315533590C800DA2BE8
:105E7000A0D376C2793C9040E8C4EAC4B0C0802187
:105E800058C2B0D0004052C2B012E064B0B000407E
:105E900048C2FA231F40CEC43F8008020130013CB3
:105EA0000F43804FC4C4B012AA5FF2C08000020248
:105EB000B0C00F0028C2A0C228C2B0D010001AC2C1
:105EC000F04384C4C04381C4B040AA5584C422D3E3
:105ED0003041B0C0030006C2B0C08021FCC1B0D0C8
:105EE0000040F6C180437AC4B012E064B0B0004014
:105EF000E8C1FA23B0C08001E0C1B0D00001DAC12E
:105F00001F4002B93FF07F00B0126066B0121A66FF
:105F10008043EEC1B0403200ECC1A0B3BCC1042448
:105F2000A0C3B6C1B012F65FB0B00300B0C1062086
:105F3000B0127264B0B00004A0C1EF27B0D000402E
:105F400098C1B012E064B0B000408EC1FA23304175
:105F5000B0128A5FA0C28AC1B0B000047CC1022422
:105F6000B0D286C122C3304180436EC1804372C12A
:105F70000F43B0128A65A0C268C1B0B000045AC114
:105F80000224B0D264C122C33041B0C080214AC1D2
:105F9000B0D0004044C1B012E064B0B000403AC19B
:105FA000FA23B0C0005032C13041B0C080012AC1D4
:105FB000B0D0000124C11F404CB83FF07F00B012A8
:105FC0006066B0121A66E0B239A20A20A0B30AC114
:105FD0000424A0C304C1B012F65FB0127264F33F90
:105FE000B0D00040F4C0B012E064B0B00040EAC0ED
:105FF000FA2330413041B090050000C1132C1F42FC
:10600000D4033F9000010E2C1F53824FD403824FC4
:10601000D603824FD803824FDA03824FDC03824FCC
:10602000DE0303433041B0B01800B6C0CB24C093A8
:10603000DCBF0A20B0B00010E8C00A24B0C01000D5
:1060400098C0B012105C623CC043C2BF8043D2C053
:10605000B0B28EC02F24E0C382C0E2B20102562447
:10606000909006C3FCC21028E0D370C09090F6C296
:10607000F0C207281F4096B73FF0FF00B0126066DD
:10608000083CB012E461053CE0C350C0B0121E6190
:106090003D20B0B0802042C00920B0D080003AC07E
:1060A000B0120E61F0438CBFB0121A66B0D08020DF
:1060B00028C02C3CE0C324C0E2B301022724B090E6
:1060C00008029EC20F2CE0D312C0809394C2072016
:1060D0001F403AB73FF0FF00B0126066073CB012B5
:1060E000E461043CE0C3F4BFB0121E61B0B0002113
:1060F000E8BF0920B0D00001E0BFB0120E61C0437C
:1061000032BFB0121A66B0D00021CEBF30413F403E
:10611000E000B0126066B040280028C23041B0C034
:106120000010B6BFA0B2B2BF4B24809316C2482065
:10613000A0C2A6BF1F409EA200184E12B0B00080A1
:1061400098BF03243E40C201073C1E40C4B63E90A7
:106150003A0202283E403A020F9E00187E41302C3F
:10616000B0B0008074BF09240E121E409ABF3EF0EA
:1061700000FF3E9000EE3E410A249090A2BF56A23E
:1061800005282F830130023C1F5303431F53809384
:106190006ABF10203F9078000D283F407800A09201
:1061A0006EB6062C90537CBFB090900176BF042849
:1061B000A0D236BF80436CBFB012606622D330419C
:1061C00022C3304180435ABFB0B000200CBF062428
:1061D000B0C080A104BFB0D00040FEBEB012E064E9
:1061E000304130413F400D00B0B00080ECBE022491
:1061F0003F401400809F04BF2A2890B3DEBE0920D0
:10620000B0D00010D4BE1F4002B6B012606690D36A
:10621000CABEC0930FBE1A24C04309BE1F40B6A118
:1062200000184E121E40E4B50D120D4E0E5E0E5EAD
:106230000E5D3D413E903A0202283E403A020F9EDA
:1062400000187E41032C1F53B01260662B3CB0C077
:10625000001086BE804384BEB0B000807CBE0D249A
:10626000B040EEEEA2BEB0C000106EBE1F4096B5AC
:106270003FF0FF00B01260663041B0C000105ABE5F
:106280001F4084B53FF07F00B0126066B0B04000A0
:1062900050BE0824B0C0180048BEB0D000403ABE7E
:1062A000B012C4613041B0B000802EBE3824B0B00E
:1062B00018002EBE1120809342BE0324B012C46188
:1062C0002E3CC09346BD0324B0D216BE283CB0D0AD
:1062D00010000EBE243C034380932CBE0B241F40B1
:1062E00026BE3FF000FF3F9000EE0724B0B00080D4
:1062F00016BE0324B012E461023C3F40EEEE8093F0
:1063000008BE0524B0B0008000BE0120083CB0C02B
:106310000080C6BDB0C01800C8BDB012C461304115
:106320008043BEBDB012C4613041B0B01000AABD00
:106330006724B0B04000AABD0820C093F2BC60241E
:10634000C043ECBCB012C4615B3CB040C201D0BDE4
:10635000B0B286BD1424B0C280BD8093B0BD0D2004
:106360008093ACBD0720B040A00FA2BDB040E803B1
:106370009EBD463C908398BD433C908390BD8093E6
:106380008CBD3E24C093A8BC15209090D4BFDABF2A
:106390000828B0D24CBDB0C0200046BDE04390BC40
:1063A0002F3CB0D010003ABDB0C0200034BDD04367
:1063B0007EBC263CD09378BC0B20B0B000201ABD28
:1063C0001F20F040030068BCB040DC053EBD183C17
:1063D000E0935CBC0B20B0B00020FEBC1120F0406C
:1063E00003004CBCB040DC0522BD0A3CF090030029
:1063F0003EBC0620809314BD03200343C04330BC41
:10640000304190B3D8BC1824B0B00001CCBC0520FA
:1064100090C3CABC80434ABF2B3CB012AC658043DA
:1064200040BF90C3B8BCB0C01800B6BCB0C080615B
:10643000A8BC8043A6BC1C3CA0B2A2BC1924B0B02E
:10644000800096BC0620A0C294BC904018BF12BF2A
:106450000F3CB012AC6590400CBF06BFA0C27EBC22
:10646000B0C018007CBCB0C080616EBC80436CBC06
:106470003041B0B0002062BC2A24B0B000105ABC39
:106480000220804356BC809372BC2120809372BC52
:106490001920809370BC1B205F406FBB3E40D864C6
:1064A000B0B0000134BC02203E40D0641F537F9046
:1064B000060001280F43C04F51BB0F5E6F4F0F5FA7
:1064C000B0122E6680433ABCB040320038BC304136
:1064D0000105040602030000030206040501000092
:1064E000B0B00040F4BB5024B0C08021ECBBB090F1
:1064F000060008BC3D2890B3E2BB0824A0B2DCBB78
:106500000E20A0B3D6BB0B24A0D2D0BB1F40FAB242
:10651000B012606690D3C4BB9040E0BBE0BB0F12EA
:106520001F40D8BB1F80D6BB2F933F412134C0935F
:10653000F3BA1A24C043EDBA1F409A9E00184E12B7
:106540001E40C6B20D120D4E0E5E0E5E0E5D3D413A
:106550003E903A0202283E403A020F9E00187E41C9
:10656000032C1F53B0126066B040460096BB0C3C33
:10657000804368BB90C364BBB0128A65809384BBC0
:106580000320B0C0807152BB30411F407CB23FF04D
:106590007F003F403200B01260663E4010200E4344
:1065A000C24E23028E10C24E2B023041B0D00040AA
:1065B00028BBB0C018002ABB3E40C8000E12B01263
:1065C000E0643E41A0B312BB0424A0C30CBB1E83F5
:1065D000032490B306BBF2233F404B00B012606629
:1065E000B0C08071F4BAB0D00040EEBA3F40640051
:1065F000A0B3E6BA0424A0C3E0BA1F830A243E4035
:106600001020C24E23028E10C24E2B028093ECBA91
:10661000EF23B0C00040C2BA3041B0122466C0437C
:10662000E9B930415F4200020F113FF00E001E4FEA
:10663000F26CB0B08000A2BA0620B0B000019ABAE5
:106640000E241E4F026DC24E23028E10C24E2B022C
:10665000B0C0004084BAB0D000207EBA22C330411E
:106660003F903A0202283F403A0280938EBA1024AB
:10667000C093C0B90420B0B268BA0A24043CB0B0D8
:1066800010005EBA05243F902D0002283F402D00E7
:10669000824FD403824FD603824FD803824FDA034E
:1066A000824FDC03824FDE033041D0B3549B16206F
:1066B000D0535CB9E09258B91628F2C07F0023028B
:1066C000B0C0802114BA804318BAB0B010000ABA22
:1066D000022030400A73F04337B9053CC09330B90B
:1066E0000224D0832AB980935ABC0224908354BCDC
:1066F000905334BA0228905330BA905328BA8093FA
:1067000040BC022490833ABCB09000F014BA022C32
:1067100090530EBAC09315B90624D0830FB9032045
:10672000F2C0400022028093C6B909249083C0B908
:106730000620F2C080000202B0C000089CB980931D
:10674000B0B906249083AAB90320B0D000088AB952
:106750008093B0B902249083AAB98093A8B9022487
:106760009083A2B990D372B9D053C0B8F0902500ED
:10677000BAB80E20C043B4B890407CB97CB912C3FB
:10678000906076B974B9904070B970B9804368B9B7
:10679000D05393B8C09372B80324D0836CB803204D
:1067A000B0C0000234B9D0537CB8F0B278B812242B
:1067B000A0D326B9C0436EB8809350B90224908309
:1067C0004AB9809326B90624908320B90320B0D01B
:1067D000000406B900184F121F4034B03FF07F008C
:1067E000C09F43B800187F410820C04339B8A0D2E9
:1067F000E8B8D05333B8D05330B8D0532AB8F09259
:1068000026B80428C04320B8F04319B8F0900A0015
:1068100017B80420B0D2C2B89053F6B8B0B0100088
:10682000B8B80720F0B04000FFB70320D0C3D59917
:10683000023CD0D3CF99001310525E060013013CE6
:1068400000130F120E1290B396B80C20F2934C0660
:106850000424F290F7004C060520C043A4B490D362
:106860007EB8003C5F409AB4DF424C06001C90B3F7
:106870006EB82124D0538AB4F0F00F0084B4F090A5
:1068800009007EB46920043CF090070074B46420D1
:10689000C0436EB490C348B83E400A000F43DF4F78
:1068A000001C011D1F531E83FA23A0D332B880435E
:1068B00076B8804374B83E413F4100130013105234
:1068C000DE050013173C003CC09357B70E240F128F
:1068D0005F422020D24F1020CE05D2532020D083FB
:1068E00041B7E04247B73F410013E2C3DC0590C324
:1068F000F2B700130F120E12B0B02000DCB709205F
:10690000F290A000CC050520C043F7B6B0D020001F
:10691000C8B75F40EDB6DF42CC05011EB0B0200025
:10692000B8B71A24D053DBB6F0F00F00D5B6F0900C
:106930000900CFB61120C043C9B6B0C020009AB735
:106940003E4009000F43DF4F011E011F1F531E83EE
:10695000FA23B0D0400082B73E413F4100131052AD
:10696000AE0300130013905384B79053D2B9C09371
:10697000E2B90524B090FF00C6B90C28043CB090E1
:10698000EA0FBCB907288043B6B9905386B70228EE
:10699000905382B7F04376B6B2B286036324905325
:1069A00054B7F2B0100001022E20C093A6B90F24F4
:1069B00040180F125F407BB61F833FF00300C04FAB
:1069C00071B6CF931C6D40183F4106200013D08351
:1069D00060B602240130001390832EB7908328B74D
:1069E000F04016004CB6C0434AB6908374B9022CEE
:1069F000908370B9B0B000806AB93324804362B923
:106A0000804360B90013C0934AB90F2440180F1295
:106A10005F401FB61F533FF00300C04F15B6CF9322
:106A2000186D40183F4107200013D05304B6F09072
:106A30001600FEB516289083D0B69083CAB6C04320
:106A4000F0B5F043EEB5905318B90228905314B93D
:106A5000B0B000800EB90524B04306B9B040FF7F46
:106A600002B90013F2B010000102CD279E3F105270
:106A70006E030013001300130013083C00130013EF
:106A8000001300130013001300130013F04274B539
:106A9000B2C010004A03B24000129203B240240276
:106AA000800392C38203B2D0100082030013001847
:106AB0004F1200184E12A2D28003B240940C9203DF
:106AC00012D350103FB5B2B24A030320F0C0800089
:106AD00033B5D0832EB57D20B2C010008203B2D072
:106AE00010004A0392C34A031F40FCB50F930224CF
:106AF0005F930B20F0E055000BB503209053E8B5F1
:106B0000683CB0C00300E0B5643C6F9328205F4050
:106B1000F3B44F105FE0EDB43FF055007F905500A7
:106B20000424B0C00300C0B5543C5F40D7B40E434A
:106B30005FB302247ED010006FB202247ED020000A
:106B40007FB0100002247ED040007FB040000724B8
:106B50007ED08000905390B5C04EAAB43A3CB0C0ED
:106B6000030084B55F409DB44F105FE097B43FF0E1
:106B700055007F9055000424B0C003006AB5293C3D
:106B80005F4081B45E407EB45FB301245ED36FB2D8
:106B900001246ED37FB0100001246ED27FB040007C
:106BA00001247ED27EE3C04E5CB4D09059B456B47A
:106BB000D04052B451B40A20B0D000021CB5D0402D
:106BC00044B444B4F040280040B4033CB0C00002D8
:106BD00008B500187E4100187F41001310520E02C4
:106BE00000130B3C203C1C3C183C143C0F3C0A3C62
:106BF000003C03438043EAB4183C03438043E2B4BF
:106C0000143C0013F040050024B40F3CF040030096
:106C10001CB40B3CC04316B4083CE04310B4053C24
:106C2000E0420AB4023CD04304B41F149053C8B4E9
:106C3000B040D007BAB4F2D0800002025E40EFB399
:106C40005F40EAB3D040E6B3E5B39053B4B45F42DB
:106C500000020F113FF00E0090B380B40C241E4FC1
:106C6000F26CC093CEB302241E4F026DC2432302C6
:106C7000C2432B021A3CC2432302C2432B023E40B2
:106C80001020B0B0005052B41020B0B000204AB470
:106C90001124B0B0800142B40D241E4FF26CB0B08C
:106CA000800036B402201E4F026DC24E23028E10A9
:106CB000C24E2B021E16001310521E020013073C78
:106CC000093C0B3C0D3C0E3C0F3C103C013C03438B
:106CD0000343001390D306B40013A0D200B40013F2
:106CE0000343001303430013034300130343001340
:106CF0000013000040021020100204084008042085
:106D00000000000004204008040810021020400287
:106D1000000001020304050001000101000101015E
:106D2000A0B3BCB3A924B0C04000B6B3A0C3B0B3F5
:106D3000D093D0AFA120B0121472B0C01800A2B38B
:106D4000F090FE00C0AF0320B0125E6F3041F090B3
:106D5000EF00B2AF0320B0127A6E3041F090EE0037
:106D6000A4AF05208043ACB38043AAB33041F09078
:106D7000FD0092AF0520B0128A5FB012105C304166
:106D80005F4081AF5E407EAF8F100FDE3F9003000B
:106D90000320B01202716E3C3F9007000320B01236
:106DA0008071683CB0B0100030B36424D0905AAF0A
:106DB00059AF60205D4052AF3DF03F000D103DF0F7
:106DC0001F000D9301201D433D90100002283D40FF
:106DD0000F0092403CAAC004824DC8041D40EC96AE
:106DE0000D100D100D100D103DF0FF0F3D903A02EB
:106DF00002283D403A023D903C00022C3D404600B6
:106E0000804D1CB3F0B0400000AF0B24B0D0100098
:106E1000D0B2B0B08080C2B22D24B0C080A1BAB2CE
:106E2000293CF0B08000E2AE2524B0D2B4B2B0B0BC
:106E30000081A6B21F24B0C080A19EB21B3C3FB00F
:106E400080000B243FC08000C04FBAAE8F10C04FEF
:106E5000B3AEB0D010008AB20D3C3FB000010A249E
:106E60003FC00001C04F9EAE8F10C04F97AEB0D252
:106E700070B20343B01244723041F090EF0085AE1F
:106E800001243041B240805A5C0132C203437E404B
:106E90004100B012486F5F424C063F4000A83E40A0
:106EA0002300B012AE723F5000021E83FA237E40D0
:106EB0004200B012486F03433E40C800B0122A6F30
:106EC0000D4F2E43B0122A6F0E4F8E100DDE0D1295
:106ED0002E43B0122A6F0C4F2E43B0122A6F0E4F62
:106EE0008E100CDE3F4000A80A430F122E43B01252
:106EF0002A6F0B4F0A5F2E43B0122A6F0A5F8F1062
:106F00000BDF0E4B3F41B012D8722F532D8301245B
:106F1000EC2F0C9A03243D4130400A733D417E40E2
:106F20004300B012486F304000F80F43D2B35D0603
:106F3000082003431F83FA235E83F8230343304072
:106F40000A735F424C0630410F120E123F4064003C
:106F50001F83FE23C24E4E063E413F413041D09337
:106F6000A5AD0B24E0939FAD5824F090030097AD9E
:106F7000AE24E09291ADBA243041D2C35C06F04019
:106F8000AA00CC963E40001C3A4014000D430C432E
:106F90003B4032001C8303201B8301203B3CD2B3C7
:106FA0005D06F827DE40A69600001E531A83F223E2
:106FB000B09055AA4CAC2E201E4048AC1E5046AC9A
:106FC0001E5044AC1E5042AC1E5040AC1E503EAC55
:106FD0001E503CAC1E503AAC1E9038AC1B2032C246
:106FE00003433F400218B012AE723F4002183D40CA
:106FF000021C3C4009003E4DB012D8722F531C8336
:10700000FA233E4055AA3F400018B012D8720343FD
:1070100032D20343D2D35C063041D2C35C063E4039
:1070200000183D4014007F4EB012F6701D83FB2304
:107030005F40E0B0B012F6705F40D9B0B012F670A9
:107040005F40D2B0B012F6705F40CBB0B012F670B5
:107050005F400EB3B012F6705F4007B3B012F67027
:107060007F403300B012F6707F403100B012F670EE
:107070007F403300B012F6705F40BCB0B012F670C3
:107080005F40B5B0B012F670B0C010005CB0B0B0E8
:10709000100046B00324B0D010004EB05F404AB09C
:1070A000B012F6705F4043B0C0939EB202243FD04E
:1070B0008000B090BF0780B0012C1FD3B012F670D3
:1070C000804326B0C04382B2D2D35C063041D2C3E3
:1070D0005C065F402CA87FE3B012F6705F4023A8E7
:1070E0007FE3B012F670D2D35C0630413F40001906
:1070F000B012AE723041E2B35D06FD27C24F4E06BC
:107100003041B0B01000D2AF37245F40FAAB3FF04F
:107110007F000F5F0F5F0B4FBF40FEFF3E211C4003
:1071200040B28F4C40213D4000013F4000F03E40C6
:107130003E213C4F3CE33CFE11243F4000F0B012A6
:10714000AE723C4000013D403E213F4000F03E4DCC
:10715000B012D8722F531C83FA230E3C1D83E923EF
:107160000F4B3F5000F03E40FEFFB012D8722F533D
:107170001E426023B012D87222D3304122C3304164
:107180005F4084AB3FF07F003F907F000A208093F8
:10719000B0B10324B012105C3C3CB0401027A2B147
:1071A000023C80439CB1B0B010002EAF32240F5F80
:1071B0000F5F0B4FBF90FEFF3E212B201E4F402143
:1071C0000D4E1D809CB106303D900A002228F043F0
:1071D0003AAE043C3DE31D53C04330AE3D900A003F
:1071E00018283D800A00804D20AF80431AAFB0D0F0
:1071F0000080E6AEB090680110AF04283D806801C1
:10720000804D04AFB040C20116AF1F40FAA5B012C6
:1072100060663041B0B01000C0AE1220C093E5AA45
:107220000E20F0900300DEAA0A20C093D9AA0720FE
:10723000F0907F00D2AA0320A0D2A6AE22D3304184
:1072400022D33041F090F700B9AA302490B394AE25
:107250002D20F043BCADD043B9ADD040A7AAB4AD0A
:10726000D0C3B0ADD0409EAAABADF0C08000A5ADFC
:10727000D04093AAA0ADD0408EAA9BAD3C40102038
:10728000B0125883C04E90ADF0400A009FADF2D0CE
:1072900040002202F040070089ADC04384ADE0D336
:1072A0003D9390D33EAEE0D3349322D33041B240ED
:1072B000805A5C0192B34401FD23B24000A5440111
:1072C000B24002A540018F43000092B34401FD2368
:1072D000B24010A544013041B240805A5C01B24036
:1072E00000A54401B24040A540018F4E0000B240CD
:1072F00000A54001B24010A544013041B240805A7F
:107300005C01B0C01000D2AD083C804338B0C0432F
:1073100036B0C04333B0F04330B03140005CB240CF
:10732000805A5C0132C20343B0400A00D0ADB04085
:107330000A00C8AD0343F043FBACB012B27BB0907F
:10734000AA550EB00920B0D010008EADB040000993
:10735000E6ADB0400024D8ADB0124E82B01226780F
:10736000B0129C7590406EAD6EADB0126E78034356
:1073700032D292D3000790C38A8D90D3848DB012FD
:107380006C740F433E401600B240185A5C0190C323
:10739000728DC0937BAC0E24B0C080213CAD804385
:1073A00040ADF2C07F0023021F83EE231E83EC2337
:1073B000C0435DACB090AF0070AD0628B0126C74E5
:1073C000804364AD804362ADB0B010000CAD0B20C3
:1073D000C09374AF0824F09003006DAF042CD05319
:1073E00067AFB012105CB0B000403AAD0424B012E8
:1073F0006E78804330ADB012CC74A0B3DCAC1624F0
:10740000A0C3D6ACB0128474B0129C759090C6AC78
:10741000C6AC05249040BEACBEACB012867AF2D0A9
:1074200080004202B0125676B0122076B012C677B3
:10743000B0120E7EB0120076B0123C80B012206DF9
:10744000B0B0100094AC9D27B012D67690B396AC35
:107450009823B012D875B0122660B0127264B012C0
:107460000264B012A662B0122A638B3F0F12F2C000
:10747000800042020F431F83FE23F2D080004202AD
:107480003F413041B0B0800150AC1F201E405AAC8B
:10749000C093B6AE02243ED08000B0B010003AAC2B
:1074A00002203ED00080B090BF078CAC022C3ED0B2
:1074B00000013EE30D4E1DE048A43EE30DFE052411
:1074C0003EE33F400019B01290F83041E2B3610250
:1074D0002624804350AC3E40C4203D400900B012F9
:1074E000227B3F4092FFB012CA7AB01286751720F5
:1074F000F093D2AB1420D093CDAB1120F090FE00CE
:10750000C6AB0E243F40C4203E40011D3D40090053
:10751000FE4F00001E531D83FB23A0D3C2AB30419E
:10752000F090EF00A3ABFB23F09003009CABF7239C
:10753000B012667AF04055007CABF040AA0077AB01
:10754000D04040A372ABD0403BA36DABD04036A33C
:1075500068ABD04031A363ABD04006AE5EABD04049
:1075600001AE59ABD040FCAD54ABB0124279B01271
:10757000087A034330410F433E4005001F83FE233A
:107580001E83FC2330413E40C5203D4005000F4393
:107590007F5E1D83FD23CE9F000030410F43F0B07E
:1075A0004000DE8C01201F53F0B08000D48C0120FD
:1075B0002FD3C04F57AA1E155E4280024E6E4E6EEC
:1075C0004E6E3EE33EF00300D2B3810201202E5204
:1075D000804E02AB1D173041B0B00020FCAA032042
:1075E00080432EAB0C3CB090080726AB0828B0C0F7
:1075F0001800EEAAB0D00040E0AAB012C461304139
:10760000B0B01000D4AA0B20E0B2D6AA0824B01261
:10761000105C0520B0D01000C0AAC0432BAD304193
:10762000E0B23E8C15203F40E8031F83FE23E0B20A
:10763000308C0E20D053D7A9B0906400D1A90A286D
:10764000C043CBA9B012105C0320B0D010008AAAAE
:10765000C043BBA9304190522007D2AA90522207C2
:10766000CEAA90522407CAAA90522607C6AAD0537F
:10767000BFA9E092BBA92628C043B5A93D4034214B
:107680009D40AAAA0000B012CA763D4036219D4016
:107690009EAA0000B012CA763D4038219D4092AAB1
:1076A0000000B012CA763D403A219D4086AA0000F3
:1076B000B012CA76804376AA804374AA804372AA25
:1076C000804370AA92D3000730412D112D11BDF0D7
:1076D000FF7F000030411F405EAA3F90AF07082C9B
:1076E00090B302AA0A20B012FC7690D3F8A9053C08
:1076F0003F90FE07022890C3ECA93041F2D08000F1
:107700000202B0402000EAA9B0C00008CCA9B0B085
:107710000008C6A9FC27B0C08001BEA9B0D00001F6
:10772000B8A91F40E0A03FF07F00B0126066B01221
:107730001A668043CCA9B0403200CAA9B0C00F007D
:107740009CA9B040409CA4A9B0C000048CA9B0B0D2
:1077500003008AA90720B0127264B0B000047AA9AD
:107760000120F53FB0C0802170A9B0D000406AA9C7
:107770008043EEABB012E064B0B000405CA9FA23E5
:10778000B01286773041B0C080014EA9B0D08000E1
:1077900048A91F4070A03FF07F00B0126066B01291
:1077A0001A66E2B301020320B0127264FA3FB0D04D
:1077B000004026A9B012E064B0B000401CA9FA2332
:1077C00090D322A93041B0B080F10EA92B201F40E8
:1077D00042A91E4042A90F9E05280F8E3F90FA0035
:1077E000012C203C034390402AA92CA9904026A9B3
:1077F00028A932C203433F408018B01266F83F40C8
:1078000080183E4055AAB01290F81E4006A92F538A
:10781000B01290F80E432F531E40FAA8B01290F801
:10782000034332D23041B09055AA56A013243F40B2
:107830008018B01266F80D433F4080183E4055AAAC
:10784000B01290F80E432F53B01290F80E432F53FE
:10785000B01290F890402CA0BAA8904028A0B6A8EA
:10786000904020A0B2A890401CA0AEA83041F2D019
:1078700040004202B01230793F408100B012CA7A13
:107880003F408180B012CA7A3F408181B012CA7AEB
:10789000B012867A3F40898CB012CA7A3F408A196A
:1078A000B012CA7A3F408B2BB012CA7A3F408C2369
:1078B000B012CA7A3F409DA3B012CA7A3F409E746C
:1078C000B012CA7A3F409FFFB012CA7A3F40A00070
:1078D000B012CA7A3F40A108B012CA7A3F40A2094A
:1078E000B012CA7A3F40A3FFB012CA7A3F40A40147
:1078F000B012CA7A3F40B103B012CA7A3F40B327F0
:10790000B012CA7A3F40B70AB012CA7A3F40DA874B
:10791000B012CA7AF2C0400042023F40C03FB012EB
:10792000CA7A3F404000B012CA7AB012087A304199
:107930000F431F83FE2330413F40E8031F83FE2394
:107940003041D2D38302B012C4793F4080003E4020
:10795000B4203D400900B0120A7BB012EA79D2C3CC
:1079600083023041F0434EA7D0434BA7F040FE00C6
:1079700046A7F040EF0041A7F04003003CA7F040CD
:10798000300037A7F040210032A7B0124279B01280
:10799000087A0F433E400A00E2B3610205201F83CC
:1079A000FB231E83F9230D3C3E40C4203D400900CB
:1079B000B012227B3F4092FFB012CA7AB012EA792D
:1079C000304130413F408181B012CA7AB0122E7AE4
:1079D000E2C26302D2D363023F409187B012CA7AF7
:1079E0003F4092FFB012CA7A30413F408182B012CC
:1079F000CA7A3F408183B012CA7AB012707AE2D25A
:107A00006302D2C3630230413F408185B012CA7A1B
:107A1000B0122E7AE2D26302D2C363023F40918752
:107A2000B012CA7A3F4092FFB012CA7A30413F404A
:107A30000E00B012CA7A8E100F4E3FD08D00B012D9
:107A4000CA7A30413F402500B012CA7A4C4E3F40BE
:107A50001300B012CA7A4C8E4F4C8F103FD08D005D
:107A6000B012CA7A30413F4092FFB012CA7A304118
:107A70000C431C8307243F401200B012CA7A3EB266
:107A8000F82722C330411E404CA63EF007000E5E90
:107A90000E5E1D4E427B1C4E447B0F4D8F103FF0FF
:107AA00000FF3FD08600B012CA7A0F4C3FF000FFB3
:107AB0003FD08700B012CA7A0F4C8F103FF000FF02
:107AC0003FD08800B012CA7A3041F2C04000420272
:107AD000C04F5C8B0E431E831324D0B34E8BFB230D
:107AE0008F10C04F4A8B0E431E830A24D0B33C8BA9
:107AF000FB235E40388BF2D04000420222D330415B
:107B0000F2D04000420222C330410C127C4E1F15BD
:107B10008C100FDCB012CA7A1E171D83F7233C416C
:107B200030410E12B012447A3E410F430E12B01291
:107B3000CA7A0C4E3E41CE4C00001E531D83F523E5
:107B40003041D9000008D9000018D9000028D90018
:107B50000038D9000048D9000058D9000068D90081
:107B60000078F240A50021011F4224010E4F3EF093
:107B7000FCFC3FF003003F900300012C1F530E5FFD
:107B8000824E2401B2B010002C01FC27B2C01000BC
:107B90002C018F1082DF24018F10B2B010002C0155
:107BA000FC27B2C010002C01C24F2001C2432101AA
:107BB0001001B013627BB013627BB013627B03438E
:107BC00032D0C0000343F2D003006A02034372D0F4
:107BD0004000034392D36201B24020006601C243D9
:107BE0006801F24060006C013F40A8611F83FE23E2
:107BF00082436E01A2C3020182436E01A2C302014D
:107C00000343A2B30201F223F24080000402F240D7
:107C10007F000602F2407F000202F2401D001802BF
:107C2000F2407F001A02D2430502F24066000702CA
:107C3000F24066000302F24066001902F24066005C
:107C40001B02F2D20B02F0D06000BB85F0400600B0
:107C5000B385C2432302F2407E002502F2D04000E9
:107C60004502F2D040004302F240E5006502C24303
:107C70006302F240C0004402F24080004202C2436C
:107C80008402F240CE008202F240CE008602F24030
:107C9000C0008502F24083008302F24003008702A5
:107CA000E042C485E042BC85F2C040002202F2D02E
:107CB00040002402F2D030002A02D2D3C005F2D014
:107CC0008000C005C243C605F2400600C705C24396
:107CD000C805D2C3C005F2D020002202F2D0200095
:107CE0002602D243DC05F2D030008A02D2D340060D
:107CF000F2D080004006C2434606F2400600470626
:107D0000C2434806D2C34006D2435C06F2D03000DC
:107D10004A02F2D080002A02D2D32006F2D06900B3
:107D20002106F2D080002006F24020002606C24341
:107D30002706D2C32006B24000485203B2401402C4
:107D40004003F24010006B02B24000994A03B2D0E7
:107D500010004A03B24010004203B24010279203C1
:107D6000B24014028003B24000C98603B2D01000B2
:107D70008603B2401402C003B2400004D203B240F2
:107D8000C000C403B240C000C603B240C000C80374
:107D9000B240C000CA03B240C000CC03B240C00031
:107DA000CE031F40609A3FF07F00824FD403824F82
:107DB000D603824FD803824FDA03824FDC03824F0F
:107DC000DE03F2D030004B02B24090FF000792D3A6
:107DD000B001B24002020207E2D21007F2D08500E1
:107DE0001107A2D300073F40001CCF4300001F53E0
:107DF0003F904423FA2B3D4000013E403E213F404E
:107E000000F0BE4F00002E531D83FB233041B0B065
:107E10004000C6A20C24B0C04000BEA2F09090006A
:107E2000E5A00C24F0905000DDA00224DC3C3041A1
:107E30005F40D4A07F90FE000624D53CF090060061
:107E4000C6A08024D03CF0905500BDA0CC20F0907E
:107E5000AA00B6A0C820B240805A5C0132C20343D7
:107E60007E404100B0121A7F5F42CC053F4000A81F
:107E70003E402300B012EA7F3F5000021E83FA23E7
:107E80007E404200B0121A7F03433E40C800B01249
:107E9000FC7E0D4F2E43B012FC7E0E4F8E100DDE79
:107EA0000D122E43B012FC7E0C4F2E43B012FC7EFE
:107EB0000E4F8E100CDE3F4000A80A430F122E43D7
:107EC000B012FC7E0B4F0A5F2E43B012FC7E0A5F9D
:107ED0008F100BDF0E4B3F41B01216802F532D83B6
:107EE0000124EC2F0C9A03243D4130400A733D419C
:107EF0007E404300B0121A7F304000F80F43D2B3E7
:107F0000DD05082003431F83FA235E83F823034320
:107F100030400A735F42CC0530410F120E12F2D08E
:107F2000400022023F4064001F83FE23C24ECE0564
:107F30003F4010271F83FE23F2C0400022023E4133
:107F40003F413041F24094001420F24031001520AE
:107F5000F2F00F001520F24033001620F2F00F006F
:107F60001620F24030001720F2F00F001720F2D058
:107F7000E0001720F2D040002202F240A0001020C2
:107F8000D2431120D242021F1220F24003001320DC
:107F90003F4011203E4007000D437D5F1E83FD23BF
:107FA0003DE3C24D18203F4064001F83FE23F24092
:107FB00009002120C24320203E4010203F400900FC
:107FC000E2B3DD0502201D83FB230D43E04E008656
:107FD0001E531F83F5230F431F830343FD23F2C06A
:107FE00040002202304122C33041B240805A5C013D
:107FF00092B34401FD23B24000A54401B24002A562
:10800000400140188F43000092B34401FD23B24069
:1080100010A544013041B240805A5C01B24000A535
:108020004401B24040A5400140188F4E0000B240CC
:1080300000A54001B24010A544013041B0B000029B
:1080400098A020245F40C09FB0C0200094A03F9023
:1080500026000624B0C0400088A0B0D0200082A036
:1080600090B37EA00E203E4012823D400F002F9E16
:1080700005242E532E531D83FA23033C1E4E02006B
:10808000C00E3041B0B0200058A00E24B0C0200077
:1080900050A00F43B0C0180048A0A0B344A00420D3
:1080A000B012D681A0D33AA03041C0435B9FC093A9
:1080B0005B9F0220D043519F3041C0434B9FD093E0
:1080C0004B9F0220D043419F3041C0433B9FE093F0
:1080D0003B9F0220D043319F3041C0432B9FF09003
:1080E0000300299F0220D0431F9F3041B012D0814E
:1080F0000520B0C01000E29FA0D2E69F3041B01230
:10810000D0810D20B0C00080D09FB0D01000D29F91
:1081100090D3CE9FA0C3CA9FB040FF0102A03041C0
:10812000B012D0810C20B0C00080AE9FB0D2B29F00
:1081300090D3AE9FA0C3AA9FB040FF01E29F304101
:10814000B012D08104203F402000B012D6813041CF
:10815000B012D08103203F42B012D6813041B0121C
:10816000D08103202F42B012D6813041B012D0818D
:1081700003202F43B012D6813041B012D0810420A9
:108180003F401000B012D6813041B012D08104209F
:108190003F404000B012D6813041B012D081002063
:1081A0003041B012D0811320B0B04000349F0F2076
:1081B000B0B01000249F0B24B0D04000249FC043D7
:1081C0006E9EB040A00F469FB040E803429F3041F2
:1081D000D093359E30410F128043449FC04F359E4F
:1081E0008F10C04F2E9EF04030002A9EF04030008D
:1081F000259EB01218830C203F410F93052090C399
:10820000E09EA0D3DC9E043C90D3D69EA0C3D29E19
:1082100030411B00EC803100AA803200BA8033006C
:10822000CA803400DA80440020814700FE805A0072
:1082300040816200508164005E8167006C8168004B
:108240007A817A008A814D009A812600A281B090BD
:1082500055AAAE9518201D40AA951D50A8951D50F1
:10826000A6951D50A4951D50A2951D50A0951D507A
:108270009E951D509C95809D9A950520B090001369
:108280008295012830413F400018B01266F80D4336
:108290003E4000133F400218B01290F80D5E3E4081
:1082A0004B003F400418B01290F80D5E3E4046006F
:1082B0003F400618B01290F80D5E3E402D003F4042
:1082C0000818B01290F80D5E3E4019003F400A18A1
:1082D000B01290F80D5E3E402D003F400C18B012D9
:1082E00090F80D5E3E400A003F400E18B01290F824
:1082F0000D5E3E40C2013F401018B01290F80D5E76
:108300000E4D3F401218B01290F83E4055AA3F4023
:108310000018B01290F8304190B3C89D1C20F04373
:10832000F09CD043ED9C3C401020B0125883C04ECE
:10833000E69CF0400A00F59CF2D040002202F0409A
:108340000700DF9CC043DA9CE0D3938290D3949DD6
:10835000E0D38A8222D330410D123F4005000D4CFC
:0E8360001D530E437E5D1F83FD233D413041C2
:10F800003F40005C3E402300B01266F83F500002CB
:10F810001E83FA2303433F40005C3C4080A87B4C9E
:10F820007E4C8E100EDBB01290F82F532D830124E6
:10F83000F62F3F4080FFB01266F83F4080FF3C400B
:10F8400000A83D4080007B4C7E4C8E100EDBB01239
:10F8500090F82F532D83F72303433F431F83FE2349
:10F860001F409CFF204FB240805A5C0192B344017C
:10F87000FD23B24000A54401B24002A540018F43E0
:10F88000000092B34401FD23B24010A54401304171
:10F89000B240805A5C01B24000A54401B24040A58C
:10F8A00040018F4E0000B24000A54001B24010A5BB
:04F8B000440130419E
:10FF80000000000000000000000000000000000071
:10FF90000000000000000000000000000000000061
:10FFA0000000000000000000000000000000000051
:10FFB0000000000000000000000000000000000041
:10FFC0000000000000000000000000000000000031
:10FFD0000000F06CB86CF06CF06CF06CF06CDC6BEA
:10FFE0005E69AE6AF06CF06C38686E6AAA66F06C96
:10FFF000F06CBE68FC72F06CF06CF06CF06C0A7324
:00000001FF
